:020000040000FA
:04000000A0EF5FF01E
:08BF3800000000000000000001
:10BF400094948294240EAC6E190EAF6E900EAB6E6C
:10BF500046D8C10853E14E0EAD6E4B0EAD6E006A71
:10BF60003ED8F86E076E3BD8F76EA96E38D8F66EDD
:10BF7000A86E35D8016E012A00EE09F0F56E2FD8B3
:10BF8000EC6E012EFBD700661FD007AC03D0040E69
:10BF90001ED818D007AE04D00C00C40E18D812D08A
:10BFA000940E15D80A00080E056E00EE0AF0080E71
:10BFB000066EEE50F56E0F00062EFBD7840E07D8E6
:10BFC000052EF5D7A694C9D74E0EAD6EC8D7A66E6E
:10BFD000550EA76EAA0EA76EA68200001200060ECE
:10BFE000026E036A046A9EAA03D0AE5000261200B5
:10BFF000042EF9D7032EF6D7022EF3D7AB9E9CD78B
:020000040030CA
:0E000000FF32F9E0FF7CFAFFFFFFFFFFFF0079
:0200000400F00A
:0400000002000128D1
:00000001FF
